:030000000207767E
:0C077600787FE4F6D8FD7581100207BD05
:0300030002006692
:10006600C0E030B20CE510700BB290B291B2928043
:0700760003751032D0E032E7
:0300130002000ADE
:01000A0032C3
:0300530002000E9A
:01000E0032BF
:03005B0002000F91
:01000F0032BE
:0300830002001068
:0100100032BD
:10064E00EFD394047480948040037F0122EF706195
:10065E00C28990000212081B64017004D2A88002A5
:10066E00C2A890000112081BFED3940374809480DC
:10067E0040037F0222EEFD7C00700553B7FEC2B828
:10068E00ED64014C700553B7FED2B8ED64024C70A8
:10069E000543B701C2B8ED64034C700543B701D2F0
:1006AE00B812080264017004D2888002C2887F00EA
:1006BE0022EF64017061C28B90000212081B64016C
:1006CE007004D2AA8002C2AA90000112081BFED3A7
:1006DE0094037480948040037F0222EEFD7C0070B0
:1006EE000553B7FBC2BAED64014C700553B7FBD28C
:1006FE00BAED64024C700543B704C2BAED64034C04
:10070E00700543B704D2BA12080264017004D28A8B
:10071E008002C28A7F0022EF6402701590000212DE
:10072E00081B64017005438F108003538FEF7F0009
:10073E0022EF6403701590000212081B640170050D
:10074E00438F208003538FDF7F0022EF64047015E8
:10075E0090000212081B64017005438F4080035302
:08076E008FBF7F00227F0222F1
:10004000750A01E4F508F509FB7A007908FF020654
:010050004E61
:1003D700EFD394077480948040037F0122120802B0
:1003E700FED394037480948040037F0222EF70440D
:1003F700EE700B90000112081BF4529352941208EE
:10040700026401700B90000112081B4293F452948E
:10041700120802FE6402700A90000112081B429340
:100427004294EE6403700D90000112081BFEF45213
:1004370093EE4294EF64017046120802FE700B902F
:10044700000112081BF452915292EE6401700B9056
:10045700000112081B4291F45292120802640270C2
:100467000A90000112081B4291429212080264038B
:10047700700D90000112081BFEF45291EE4292EFAC
:1004870064027046120802FE700B90000112081BEE
:10049700F452955296EE6401700B90000112081BFE
:1004A7004295F452961208026402700A90000112F3
:1004B700081B429542961208026403700D900001D2
:1004C70012081BFEF45295EE4296EF640370461233
:1004D7000802FE700B90000112081BF452B152B2D1
:1004E700EE6401700B90000112081B42B1F452B286
:1004F7001208026402700A90000112081B42B142FE
:10050700B21208026403700D90000112081BFEF47A
:1005170052B1EE42B2EF64047046120802FE700B4D
:1005270090000112081BF452B352B4EE6401700B31
:1005370090000112081B42B3F452B412080264027D
:10054700700A90000112081B42B342B412080264F9
:1005570003700D90000112081BFEF452B3EE42B473
:10056700EF64057046120802FE700B900001120836
:100577001BF452C952CAEE6401700B9000011208B5
:100587001B42C9F452CA1208026402700A900001A1
:1005970012081B42C942CA1208026403700D900078
:1005A7000112081BFEF452C9EE42CAEF64067046F8
:1005B700120802FE700B90000112081BF452CB5276
:1005C700CCEE6401700B90000112081B42CBF45271
:1005D700CC1208026402700A90000112081B42CB79
:1005E70042CC1208026403700D90000112081BFE32
:1005F700F452CBEE42CCEF64077049120802FF7E3B
:1006070000700B90000112081BF452E152E2EF64F4
:10061700014E700B90000112081B42E1F452E212E6
:1006270008026402700A90000112081B42E142E2CC
:100637001208026403700D90000112081BFFF452A8
:07064700E1EF42E27F002217
:10001E00750904E4F508FB7A0079087F031203D70B
:10002E007509077508037F011203D7C290C291C2EA
:01003E00922F
:01003F00229E
:0D00860012001E120040120880D2AF80FE52
:03000600011000E6
:03000B0002089E4A
:0B089E00C0E0E51060021510D0E03251
:03001B00020011CF
:0100110032BC
:0300630002001286
:0100120032BB
:03009B000200164A
:0100160032B7
:0300A30002001741
:0100170032B6
:1000A600AD07EDD394047480948040037F0122ED64
:1000B600600302017BC28C90000212081B6401706F
:1000C60004D2A98002C2A990000112081BFED39493
:1000D600037480948040037F0222EEFF7E00700549
:1000E60053B7FDC2B9EF64014E700553B7FDD2B9DF
:1000F600EF64024E700543B702C2B9EF64034E7057
:100106000543B702D2B9120802FEC3940374809461
:100116008040037F0222E58954FC4EF58990000356
:1001260012081BFF7E0064017003538E7FEF4E7032
:1001360003438E80EF64024E7005438904800353A7
:1001460089FB90000412081B64017005438F01802F
:1001560003538FFE900005120848E5F0F58C9000D9
:1001660005120848F58A90000712081B6401700200
:10017600D28C7F0022ED64016003020248C28E9099
:10018600000212081B64017004D2AB8002C2AB905D
:10019600000112081BFED394037480948040037FF1
:1001A6000222EEFF7E00700553B7F7C2BBEF640173
:1001B6004E700553B7F7D2BBEF64024E700543B7D6
:1001C60008C2BBEF64034E700543B708D2BB1208E2
:1001D60002FEC394037480948040037F0222EEC41F
:1001E60054F0FFE58954CF4FF58990000312081BA0
:1001F600FF7E0064017003538EBFEF4E7003438E83
:1002060040EF64024E700543894080035389BF90D6
:10021600000412081B64017005438F028003538F8C
:10022600FD900005120848E5F0F58D9000051208CE
:1002360048F58B90000712081B64017002D28E7F6E
:100246000022ED6402707C538EEF90000212081BB0
:100256006401700543AF04800353AFFB90000312A3
:10026600081BFED394027480948040037F0222EE22
:10027600FF7E0064017003538EFBEF4E7003438EC6
:1002860004EF64024E7005438E088003538EF79088
:10029600000412081B64017005438F048003538F0A
:1002A600FB900005120848E5F0F5D6900005120807
:1002B60048F5D790000712081B64017003438E109F
:1002C6007F0022ED6403707C53D1F7900002120880
:1002D6001B6401700543AF20800353AFDF9000031A
:1002E60012081BFED394027480948040037F02227E
:1002F600EEFF7E006401700353D1FDEF4E700343A1
:10030600D102EF64024E700543D104800353D1FB42
:1003160090000412081B6401700543D10180035349
:10032600D1FE900005120848E5F0F5D490000512BC
:100336000848F5D590000712081B6401700343D1E5
:10034600087F0022ED640460030203D453D17F903A
:10035600000212081B6401700543AF40800353AFCF
:10036600BF90000312081BFD7C00D3940274809496
:100376008040037F0222ED64014C700353D1DF906D
:10038600000312081B700343D12090000312081BC0
:100396006402700543D140800353D1BF900004121C
:1003A600081B6401700543D110800353D1EF900000
:1003B60005120848FDACF0ECF5D2AF058FD39000DE
:1003C6000712081B6401700343D1807F00227F025D
:0103D6002204
:10088000E4F508F509750A01F50BF50C750DD4753D
:0E0890000ECD750F01FB7A007908FF0200A65D
:10078200020086E493A3F8E493A34003F68001F207
:1007920008DFF48029E493A3F85407240CC8C33378
:1007A200C4540F4420C8834004F456800146F6DF47
:1007B200E4800B0102040810204080900006E47ED1
:1007C200019360BCA3FF543F30E509541FFEE4933C
:1007D200A360010ECF54C025E060A840B8E493A303
:1007E200FAE493A3F8E493A3C8C582C8CAC583CA2E
:1007F200F0A3C8C582C8CAC583CADFE9DEE780BEE6
:0100090000F6
:10080200BB010689828A83E0225002E722BBFE02F4
:09081200E32289828A83E4932227
:10081B00BB010CE58229F582E5833AF583E0225092
:10082B0006E92582F8E622BBFE06E92582F8E222DC
:0D083B00E58229F582E5833AF583E49322F6
:10084800BB0110E58229F582E5833AF583E0F5F0EE
:10085800A3E0225009E92582F886F008E622BBFECB
:100868000AE92582F8E2F5F008E222E5832AF58311
:08087800E993F5F0A3E99322D6
:00000001FF
